:10000000A42A82004F347C2957345B345F345D343A
:1000100072297C294D345134553459347B34FF34A2
:100020007C297C2906293F347C290229DF34FD34D0
:100030007C297C297C299D34BD34BF34DD34FB34DC
:100040007C297C2999349B34BB34DB34F734F93474
:100050007C297C297F349734B934D734D934F534AA
:100060007C297C2993349534B534B734D534F334B2
:100070007C297C297C299134B334D334F134EF3496
:100080007C297C298F34B134D134CF34EB34ED3436
:100090007C297C298D348B34AF34AD34CD34E934B4
:1000A0007C297C297C29AB347C29CB34E7347C291E
:1000B0007C2967293D347734C9347C29A9347C29CB
:1000C0007C297C299F347C297C297C297C297D34CE
:1000D0007C297C29C5347C29A53485347C297C295C
:1000E0007C29E1348734C334A334A1348334753498
:1000F0005F297C294334C1346B34453481347529FC
:100100007C297C297C297C29533423297C297C293E
:100110007C297C297C297C297C297C297C297C29B7
:100120007C297C2909297C297C2900297C297C2996
:100130007C297C297C297C297C297C297C297C2997
:100140000C297C297C297C297C297C297C297C29F7
:1001500012297C297C297C297C297C297C297C29E1
:1001600018297C297C297C297C297C297C297C29CB
:100170007C297C297C297C297C297C297C297C2957
:100180007C297C297C297C297C297C297C297C2947
:100190007C297C297C2947347C297C297C297C2961
:1001A0007C297C297C297C297C297C297C297C2927
:1001B0007C297C297C2979347C297C297C297C290F
:1001C0007C297C297C297C297C297C297C297C2907
:1001D0007C297C2937297C2961342D297C297C299B
:1001E00063347929733465347C29633467347C291A
:1001F0007C297C297C2941297C2923294B297C299C
:100200009E1F7C291A141A1A1A1039349E1E0E29A0
:1002100037349E1E142935349E1E37349A141A1A08
:100220009A1033349E1E35341A151A1A1A113134A5
:100230009D1C7C291A1E00343330B6219130EB21ED
:100240003230B62100341D1F7C291A1E0034313093
:10025000B621CD30EB21303021291D1D7C291A1EFD
:1002600000343D30B6216130EB213C3021299D1D09
:100270007C291A1E00343D30B6216330EB213C301E
:1002800021299D1E7C291A1E00343D30B62165307F
:10029000EB213C3021291D1E7C291A1E00343D30E3
:1002A000B6216730EB213C3021291E1C7C291A1E07
:1002B00000343930B6219930EB21383021291E1E07
:1002C0004B341A1E003402309B06972100349E1DC9
:1002D0007C291A1E003404309B0697213B301B1DDD
:1002E000FE3921291E197C2941349E187C299A1235
:1002F00000349D1F7C29413494092E30B6211E30D4
:1003000091001A1A11119A1991109A1E911111083F
:10031000B62114089100910D11081E39B621940ED2
:10032000940D14081E39212901301B069B00ED3065
:10033000F2212B220508F8391B0485001B08F22145
:100340002B2AA3210030962125309100AA21910B60
:10035000A6290800FF3092006400920BAD29080026
:1003600090000F020319080010088F0090000A3057
:10037000A52108309100A300901B8515901F8511C1
:100380000A30AB2105120A30AB2105160A30AB2129
:10039000900D910BBC298316851583129101920152
:1003A000851DDA296400910BD029920BD0291A1BE4
:1003B0000800E6291A1B080091018519E129910B13
:1003C000DD2985158316851183120800E121910A24
:1003D000A30BC02908009700B6211708FE39B621E3
:1003E0001708080094009501861400000610831673
:1003F00086100000061083120830910083168614C0
:1004000083128618012A14180614141C0610940C62
:100410000318950A861C0A2A910B012A86180E2AAF
:1004200015180610151C0614861C142A8618162A80
:100430000614861C192A83160614831286181E2A8F
:10044000861C202A0830AB21861083168610831262
:100450001430AB21080096011A169A1186148316DF
:1004600086148312861C3D2A6400061B322A9A1EBB
:10047000322AA11FDF2BA1138C2A861C3D2A0830AB
:1004800091008618412A940C06189417061C9413A0
:10049000861C482A910B412A86184C2A861C4E2A13
:1004A0008618502A861C522A88221430AB2116083E
:1004B00003195C2A96032E2AE130140203197B2AC1
:1004C000E030140203197F2AF03014020319812A44
:1004D0009A1D732A1230140203192B2A5930140260
:1004E00003192B2A080083301402031D08009A15F3
:1004F0000330940008005521073096002C2A9A15E5
:100500002E2A1A122E2A86148316861483120800A5
:10051000861083168610862A0F30B6211A170F30E0
:10052000B6211630930085199C2A910B932A920BC1
:10053000932A9421930B932A051283160611831292
:10054000FF30A521A11FD12B1C2307309A008F015A
:10055000103038239D0039239E0039239F00392312
:10056000A0003923A100061CB32AFF30F221073076
:10057000A121F3309F21FF309F211E1BC12AA11F03
:10058000D12B0230B6210230B6219A161A0807394B
:1005900003198C2A9A1EEB2A2B221A19DC2A1E1BFD
:1005A000D62AC6239A1BD62AA1138C2A9A18DC2A8B
:1005B000073014020319412B941FE02A7C21C62A1C
:1005C000140A9A19803E0120003E0319C62A1A1EF9
:1005D000FE39B021C62A06129C01A20191014030C9
:1005E000920883226400861CFC2A910BF22A920B4B
:1005F000F22A88229421182B7C23003E031D182BFD
:10060000392314020319A20A5A301402031D142BB1
:1006100022081C02031DEB2AFF3094007C211B10D2
:1006200097219A160616C62A10301C020319EB2AC7
:100630001C0894007C21EE2A8312183085001830A3
:100640008600831681138501C73086008312080057
:1006500088001C0889009C0A8316081555308900FB
:10066000AA3089008814081E332B880183120800E1
:100670009C001C0889009C0A831608148312080831
:1006800008001A123330EB213130EB214330EB21DB
:100690007C239823163014020319532B1E301402A6
:1006A00003196B2BA42A9C017C23663014020319C6
:1006B000672B9823140828235A3014020319462B59
:1006C0000F301C02031D542B5A309400592B1C0868
:1006D000031D9C03542B10309C007C239E23980008
:1006E000980E98237C239E231804282398231430E3
:1006F0001C02031D6D2B462B2B22941B912B1A1EC3
:10070000912B9A19912B91015930942358309423AD
:1007100011309423123094231430942311080319B8
:1007200000349A1E01347C2B14020319910A08002C
:10073000140A0120003E03190800EB2991019201DF
:100740001630BD231E30BD232630BD232530BD23EA
:100750002E30BD233630BD233D30BD233E30BD237A
:100760004630BD231C30BD233230BD232130BD2394
:100770002330BD232430BD232B30910A14020319EA
:10078000C32B120808001108920008009A171A08D3
:10079000F7381F02031D08002008140203199A13DA
:1007A0000800A11314309C00210828238611861606
:1007B000E6232B221A1ED92BC6239A1BD92BA1174D
:1007C00014309C0021082823E623A42AE923061FCD
:0607D000E62B8030A52994
:084000000000010001000900AD
:02400E00F73F7A
:104200001C003A00430034001C005A00FF00FF006D
:10421000FF00FF00FF00FF00FF00FF00FF00FF00A6
:0A422000FF00FF00F7007600FF002A
:00000001FF
